:020000040800F2
:1000000088050020D900000835200008751E00086A
:1000100000000000000000000000000000000000E0
:100020000000000000000000000000007F20000829
:1000300000000000000000007D2000088120000872
:10004000EB000008EB000008EB000008EB000008E4
:10005000EB000008EB000008EB000008EB000008D4
:1000600000000000EB000008EB000008EB000008B7
:10007000EB000008EB00000800000000EB000008A7
:1000800000000000EB00000800000000000000007D
:10009000EB00000800000000EB000008EB00000887
:1000A000EB000008EB000008EB0000083D2600080C
:1000B000EB000008EB00000800000000000000005A
:1000C0000448854600F0EEFB00480047A12F0008D9
:1000D000C046C046880500200448804704480047C1
:1000E000FEE7FEE7FEE7FEE7FEE7FEE7F520000895
:1000F000C100000830B50B46014600202022012433
:1001000009E00D46D5409D4205D31D469540491B4B
:100110002546954040191546521E002DF1DC30BD94
:10012000F0B51FB40646002082B005464024019178
:1001300000901BE0019922460F46304600F0BAFAC3
:10014000049A059B801A994110D3104619462246FD
:1001500000F0A0FA361A8F410197224601200021B3
:10016000009F00F097FA38184D4100902046641E19
:100170000028DFDC019B00982946324607B0F0BD1D
:10018000D2B201E00270401C491EFBD2704700222F
:10019000F6E710B513460A4604461946FFF7F0FF86
:1001A000204610BDF8B502464A40D40F42004B002D
:1001B00052085B089A4202D20246084611464A009B
:1001C00023D0C30D4A00DDB2120EAD1A202D35DA50
:1001D00049020126490AF6058A19002C00D052422C
:1001E00020214F1B1146B9402A411018C20D9A42D6
:1001F00021D0002C17D0012D08DCDA05801AD20F8F
:100200008019D207DBB200F081FAF8BDDA05801A56
:10021000012340001B06C01880185A428018CA0FDC
:100220001043490007E04908C2071143DA05801A64
:1002300080194008801800F061FAF8BD61000122C1
:10024000511A001BF7E70122D2075140AAE7012209
:10025000D2075040A6E7024670B54A40D30FDB07ED
:1002600040002DD04A002AD0010E140E00021202C6
:100270000919400A520A8418E50104465443000A49
:10028000120A2E045043A4194219200CC543AA187F
:10029000120C0125AD03521C521912047F3924049B
:1002A00000D0521C104301D44000491EC2B20C06BB
:1002B000C0092018401C4008802A02D003E000201A
:1002C00070BD40084000002900DA0020184370BDCE
:1002D000420005D04200120E52428A4201DB002049
:1002E0007047C90508187047F0B5074608465840DA
:1002F00087B0C00F049048000E46590040084908D6
:10030000BC1A884105D2384631461E4617460B4670
:1003100002465800400810434DD0300D0390400570
:100320005900400D490D0590401A0290402873DA9B
:1003300018030121000B090508430190049800925D
:10034000002806D01146019A4942002090410091B0
:100350000190029840210A1A0199009800F09AF938
:1003600005460C466B4607CB00F0B5F9C019714144
:10037000039A0E0D0023D71756401A467A401643AB
:1003800044D0049A002A2DD0029A012A039A15DC3F
:100390001205C01A914101263605001C7141D20F89
:1003A000059ED2070093019202962A46234600F04A
:1003B000F3F907B0F0BD38463146FAE71605234A8F
:1003C0000F46B218C01AB74101210905001C4F4160
:1003D00000187F41114618187941E20F10436D193A
:1003E000644113E0E2076D0815436408C207144333
:1003F000039A01261205C01A91413605001C71416D
:10040000CE07400830434908C01851412A462346C8
:1004100000F0B5F9CDE7FFE7049801224000C117CD
:10042000121A00238B4104983146C417381AA1418F
:10043000EEE730B40124E407634030BC54E730B445
:100440000124E407614030BC4EE700000000E0FFFB
:10045000F0B51FB488B00B99099800244840099959
:10046000C00F490049080991C0070B990090490045
:1004700049080B9109990898A64608431CD00B9986
:100480000A98084318D0099801244000420D4800FA
:10049000410D099824050003000B204309900B9897
:1004A0000003000B20430B9050181C4940180022F9
:1004B00001901446104605E0002001460DB0F0BD45
:1004C000032801DA034600E003239C46C11A0AAE62
:1004D0000AE05F0008ADED5B4F00F75B7D4300274E
:1004E000AA187C41491C5B1E6145F2DD410004AB4A
:1004F0005A522104120C0A43240C401C0828DFDB4A
:10050000019802900099704601910090059B049A11
:100510000799069800F040F9D0E700000DFCFFFFB6
:10052000F0B50C465C4085B0E40FE40703944C0042
:100530000026640859009446490802460296224360
:1005400021D062460A431ED06200570D4A000E03B6
:100550002303550D012402462C492405781B1B0B4F
:10056000360B401823432643614600901C46501A20
:10057000B44103D30098401C009002E09218009808
:100580005B41002803DA0020014605B0F0BD0020E1
:10059000012109050746864611E064461D46141BE5
:1005A000B54106D36546521BB341744607430C431D
:1005B000A646CD0740084908284392185B410546E6
:1005C0000D43EAD11046184313D0604619465040F7
:1005D0007140084306D06046101AB34106D201228A
:1005E000002306E000220123DB0702E00122D243C0
:1005F0005310009874460105381C6141029C039D0C
:100600000019694100F0BBF8BFE70000FD030000DE
:1006100010B500229623114600F078F810BDC20FE5
:10062000D207400040080BD0C10D0723DB01C918D9
:1006300040020905400A1143C208400711437047B0
:10064000002001467047CB0FDB07490010B5490871
:1006500002460A4307D00A0D07240903E401090BE7
:10066000121B002A01DC002010BDC900440F0C43FE
:10067000C100E018D205801800F040F810BD00005D
:100680000122D207002800DB101A002900DB511AD2
:100690008842704710B5202A04DB0146203A914079
:1006A000002010BD914020239C1A0346E3401943CB
:1006B000904010BD10B5202A04DB0846203AD040F7
:1006C000002110BD0B46D340D0402024A21A9140F7
:1006D0000843194610BD10B5202A06DBCB17084683
:1006E000203A1041C1170B4306E00B461341D0409E
:1006F0002024A21A91400843194610BD002904DAAB
:10070000401C490001D140084000704770B40024EB
:10071000050C05D11024000402D1002921D0112498
:10072000050E01D100020834050F01D10001241D7E
:10073000850F01D18000A41C002801DB4000641C4F
:10074000002908D020252E1B0D46F540A14000D0E1
:1007500001212943084301061B1B000ADB1D02D5AA
:10076000002070BC7047DB05181880180029F8DAE3
:10077000401C4900F5D170BC40084000704710B5DE
:10078000002B08DA0024401C614192185B411A4397
:1007900001D14008400010BDF0B51FB482B005463D
:1007A0000C0003D0084601F061FF02E001F05EFF9B
:1007B00020300246009021462846FFF76BFF049B3D
:1007C000059A04460F4618431143084314D01846AF
:1007D00010431BD0009840210A1A18460599FFF7CC
:1007E00069FF05460E46009A05990498FFF752FFE7
:1007F000084305D0012004E02046394607B0F0BD8B
:100800000020C11705430E432C43374300990E982F
:100810006305401A7905E40A00220C43FD0A0A30F8
:1008200002D500200146E9E70105101969410C9C39
:100830000D9D00196941FFF7A2FFDFE74A00090398
:100840000123090B1B0519430A4B10B5520D9A429F
:1008500002DA0020014610BD064B34339A4203DC15
:100860009A1AFFF727FF10BD034BD218FFF712FFAC
:1008700010BD0000FF030000CDFBFFFF10B50029F5
:1008800004DB0124E40740428C412146002B04DBB9
:100890001C460123DB075242A341994200D19042FA
:1008A00010BD0000064C0125064E05E0E36807CCAC
:1008B0002B430C3C98471034B442F7D3FFF704FCA9
:1008C000FC3000081C31000838B5044606480549CC
:1008D0000068FFF70FFC604300E0401E0090002816
:1008E000FBD138BD40420F0018000020F8B5044687
:1008F000006881688907890F012902D10168C90749
:1009000022D18168114A10261140012500290ED1FB
:100910008168294381600120FFF7D6FF00F0FAFAD1
:1009200007460CE000F0F6FAC01B0A2807D9606DF4
:1009300030436065A06D2843A0650120F8BD2068A4
:100940000068C043C007EDD10020F8BD170000804B
:1009500070470000F8B506460D464036317C012947
:100960000DD00121317401688A68520709D5416DA3
:10097000202211434165002030740120F8BD02207F
:10098000F8BD174B6A68D80547109A42154C8A6A19
:100990002B6812D05B035B0B1A438A6229684903F8
:1009A00005D5A1680143A1600A20FFF78DFF2868E3
:1009B000800312D5A06838430EE05B035B0B9A43BB
:1009C0008A622968490302D5A1688143A160286829
:1009D000800302D5A068B843A06000203074F8BD41
:1009E0000110000000270140406D70470068006C56
:1009F0007047000070B5040006D0606D26460025E3
:100A00004036002802D006E0012070BDA56535748F
:100A1000204600F0D3F8606DC00603D421688868D2
:100A2000400705D5606D1021084360653574EBE71C
:100A3000606DFF2201329043022210436065886896
:100A40008207920F5B48012A02D10A68D2072BD194
:100A5000032362689B079A4205D05B429A4202D008
:100A60005B009A4209D10A69920092080A612168E2
:100A70000A6963681A430A610CE00A6992009208E5
:100A80000A6181680F2292049143816081686268E3
:100A9000114381602168CA6818239A43CA6021689B
:100AA000CA68A3681A43CA6081680122520691434A
:100AB00081608168A28E520611438160206881683E
:100AC000C90004D4816801221207114381602068A3
:100AD000C168394A1140C1602069E168022825D007
:100AE00000200143204620300278037B52035B0044
:100AF0001A431143226B1143A26992031143E26925
:100B0000D20311432268D3681943D160616A0A464F
:100B1000FF3AC23A05D0A26A11432268D36819434A
:100B2000D16042780121012A02D00BE00420D8E7ED
:100B30000078002823D0606D202210436065A06DEE
:100B40000843A065E06B012820681FD00169C90730
:100B500003D0016949084900016120684169C90859
:100B6000C900416120684169A26B11434161A565DB
:100B7000606D80088000401C6065002070BD2068AA
:100B8000C26801231B041A43C260DBE70269FF232A
:100B90009B009A43026120680269236CA66C1A4389
:100BA000636C33431A430261206802690A4302619D
:100BB000D3E70000002701401902FEFF10B586B000
:100BC000044614216846FFF7E2FA0E49206888427D
:100BD00016D10D48416B421511434163C16A012290
:100BE0001143C162C06A6946104005901020009010
:100BF00003200190002002900520000700F0C8F8B3
:100C000006B010BD0024014000100240F8B50446B3
:100C10004069254640350E4608280BD02068C0683C
:100C2000C00709D0606D202108436065002028744A
:100C30000120F8BD082700E00C2700F06BF90090B8
:100C400011E0701C0FD0002E05D000F063F9009960
:100C5000401AB04207D9606D042108436065002046
:100C600028740320F8BD206800683842E9D0606D20
:100C700001214902084360652068C16809058A0F9F
:100C80000C21002A1BD12022125D002A17D10268F4
:100C9000120714D5826853070122002B08DB436832
:100CA0008B434360606D130298431043606506E018
:100CB000606D202318436065A06D1043A065A06996
:100CC000002801D1206801600020F8BD70B50446FD
:100CD000216800208968490721D425464035297CB0
:100CE00001291CD001212974E169012904D0204681
:100CF000FFF7FCFD002811D1616D0A4A1140FF2267
:100D00000132114361650021A165297422681C210B
:100D1000116021688A6804231A438A6070BD02202A
:100D200070BD0000FEF1FFFF70B5002401462031C8
:100D30004A79022A03D00421C163012418E0026821
:100D400013680E25AB431360026813685B085B00F1
:100D50001360436C1C221340012215469D40036C16
:100D60005D604A7100220A71816B002900D08847BA
:100D7000204670BD70B5044600F0CCF80546601CF6
:100D800000D0641C00F0C6F8401BA042FAD370BD2E
:100D9000F8B500230124A2E027469F403A4070D0D6
:100DA0004D68022D01D0122D14D1DD08AD002D1893
:100DB00000952D6A5E07AC46F50E0F26AE46AE4096
:100DC0006546B543AC460E697546AE4065462E4352
:100DD000009D2E624D68012D05D0022D03D0112DEE
:100DE00001D0122D16D185680326AC465D00AE46B3
:100DF000AE406546B543AC46CE687546AE406546E6
:100E00002E43866046680D79BE43ED06ED0F9D408A
:100E10003543456006685F000325BD40AE46AE43DE
:100E20000D79B446AE07B60FBE4065462E43066048
:100E3000C6687546AE438D68BD403543C5604D6894
:100E4000ED004BD5294D6E6B26436E639E08284DF1
:100E5000B6007519AC46AD689E07360F0F27B74030
:100E6000BD4305273F07B84201D1002715E0214FB8
:100E7000B84201D1012710E01F4FB84202D102272A
:100E80000BE02BE01D4FB84201D1032705E01C4FBA
:100E9000B84201D1052700E00627B7402F43654639
:100EA000AF60184D2E684F689643FF0300D5164378
:100EB0002E606E684F689643BF0300D516436E6080
:100EC000AE684F689643FF0200D51643AE60EE68E9
:100ED0004F689643BF0200D51643EE605B1C0A685C
:100EE0001546DD4000D057E7F8BD00000010024075
:100EF000000001400004005000080050000C0050A9
:100F0000001C005000040140002A01D0816170479C
:100F1000816270470148006870470000140000209B
:100F200070B5024640325378202B1CD11378012B28
:100F300019D00123137024245470046825689D433C
:100F40002560046825681E03B5432560046825688C
:100F50000D4325600068016819430160202050702E
:100F60000020107070BD022070BD70B50246403286
:100F70005378202B1BD11378012B18D00124147027
:100F80002423537003681D68A5431D6005682B6802
:100F90000F263602B343090219432960006801682D
:100FA00021430160202050700020107070BD02208D
:100FB00070BD000070B5040006D025464035687845
:100FC0000026002802D005E0012070BD2E702046CA
:100FD00000F04AF824206870206801684908490038
:100FE00001600F2160680906884321680861216853
:100FF0008A680120C00382438A60E1680129A168F0
:1010000008D021229202114322689160E1680229EE
:1010100002D005E00143F7E701212268C9025160CF
:1010200021684A680F4B1A434A602168CA688243A4
:10103000CA60616920690843A169090208432168FF
:10104000C860216AE0690843216808602068016877
:101050000122114301606664202068702663AE702F
:10106000002070BD0080000210B586B00446142137
:101070006846FFF78CF81149206888421BD1104C54
:10108000E16A02200143E162E16A01400320059127
:101090008002009012200190012002900320039012
:1010A0000620049069460748FFF772FEA06B0121F5
:1010B00089050843A06306B010BD00000058004039
:1010C000001002400004005002480168491C016001
:1010D000704700001400002010B508480024016883
:1010E000402211430160204600F00AF8002801D098
:1010F000012401E000F01CF8204610BD0020024051
:1011000070B5054609487D210024C9000068FEF736
:10111000F1FF00F0F9FB002801D0012404E00022D7
:101120002946501E00F01AF8204670BD1800002015
:101130000448416B012211434163816B0204114356
:101140008163704700100240C106C90E012088402B
:10115000014908607047000000E100E010B500F0B0
:101160006BFF10BDF8B504460078544D800672D56B
:10117000524E0027403EB06BC00004D4B06BA905AE
:101180000843B06301274E480168C90511D40168BE
:10119000821511430160FFF7BDFE009005E0FFF7E7
:1011A000B9FE0099401A642837D845480068C00540
:1011B000F5D532680321090560680A400140914273
:1011C00008D08103890F032904D13168890301D52F
:1011D0000120F8BD2A69032109040A4022D00840F1
:1011E00090421FD0207880061CD528692A69884340
:1011F0000121C9040A432A612A698A432A612861B4
:10120000C0050FD5FFF786FE009008E0FFF782FECD
:101210000099411A2B48814201D90320F8BD286961
:101220008005F3D561688803800F032805D13268F3
:101230000005824301400A43326028690322616845
:101240001204114008432861002F04D0B16B012023
:1012500000078143B1632078C00705D0E868A16822
:10126000800880000843E8602078800705D5E8689A
:101270000C218843E1680843E8602078400706D5E0
:10128000E86803218902884321690843E8602078DF
:10129000000706D5E868032109038843616908430C
:1012A000E8602078000606D5E868032189048843B1
:1012B000A1690843E8600020F8BD0000401002402A
:1012C0000070004088130000F8B50E4605007DD080
:1012D00053480068C007C00FB0420AD250480168A6
:1012E00049084900314301600068C007C00FB0429F
:1012F00071D128784B4C800705D5E068F0218843F0
:10130000A9680843E0602878C00752D068680228BE
:1013100017D0032818D02168012818D08905002982
:1013200059DAE168890889000143E160FFF7F2FDBD
:1013300069680746022912D003291CD0012926D04A
:1013400033E021688903EAE721688901E7E7490773
:10135000E5E7FFF7DFFDC11B3348814223D8E06892
:101360000007800F0228F4D123E0FFF7D3FDC11B53
:101370002D48814217D8E0680007800F0328F4D178
:1013800017E0FFF7C7FDC11B274881420BD8E06873
:101390000007800F0128F4D10BE0FFF7BBFDC11B54
:1013A0002148814201D90320F8BDE0680007800F81
:1013B000F3D11B480168C907C90FB1420DD90168B3
:1013C0004908490031430160006800E003E0C007BC
:1013D000C00FB04201D00120F8BD2878400706D5E3
:1013E000E068072109028843E9680843E06028783B
:1013F000000707D5E0680721C90288432969C900A9
:101400000843E06000F036F8E168084A0906090F71
:10141000515CC840064908600020FFF771FEF8BD26
:10142000002002400010024088130000D83000085D
:1014300018000020044805490068C968044A4905A5
:10144000490F515CC840704718000020001002404E
:10145000F1300008044805490068C968044A890455
:10146000490F515CC840704718000020001002402E
:10147000F130000810B5184AD1680C200840042843
:101480000BD0082810D00C2810D050680004410F51
:101490000120C003491C884010BD1068C00601D55A
:1014A0000E4810BD0E4810BD0E4810BD88020E4BF0
:1014B000000F185C0902D368890F491CDB0301D5B2
:1014C000084A05E01268D20601D5044A00E0044A41
:1014D0005043FEF70FFE10BD0010024000093D0012
:1014E0000024F40000127A00E8300008FEB5050080
:1014F0007ED0FE4CE7680C20E6680740012000041F
:1015000006402878C00747D0082F05D00C2F0AD1F5
:1015100001200004864206D1206880033CD568681B
:101520000028E5D038E0012069680004814203D139
:1015300021680143216011E0052301221B0492046C
:101540009942216802D111432160F1E78143216072
:10155000216801400091206890432060686800285D
:101560000DD0FFF7D7FC009005E0FFF7D3FC009902
:10157000401A64287AD820688003F6D50CE0FFF77B
:10158000C9FC009005E0FFF7C5FC0099401A6428EB
:10159000F0D820688003F6D42878800755D5092331
:1015A000E868042F0DD00C2F01D1002E09D000289F
:1015B0003BD02168994301432160FFF7ABFC06460D
:1015C00027E02168490701D5002891D061681F22D2
:1015D000120291432A691202114361602168994302
:1015E00001432160FFF746FFE16809060A0F00E0AA
:1015F00079E1BF49895CC840BE4908600020FFF717
:101600007FFD002872D120E0FFF784FC801B0228B8
:10161000B0D820684007F7D560681F2109028843C9
:1016200029690902084360600FE020684008400013
:101630002060FFF76FFC064604E0FFF76BFC801BA1
:10164000022897D820684007F7D42878C0065FD5CD
:10165000002F0CD0A869002849D02068FF21013153
:1016600008432060FFF756FC06462DE0C0E02068E6
:10167000800502D5A8690028A7D060680721490322
:101680008843296A084360606068297F0002000A75
:10169000090608436060286A410B0120C003491C09
:1016A0008840E16809060A0F9149895CC840914960
:1016B00008600020FFF724FD002817D128E0FFF77D
:1016C00029FC801B0228A3D820688005F7D5606814
:1016D000072149038843296A084360606068297FBD
:1016E0000002000A09060843606011E0E1E0216899
:1016F000FF20013081432160FFF70CFC064604E027
:10170000FFF708FC801B022872D820688005F7D4F8
:101710002878794E000724D568690028306910D0F0
:10172000012108433061FFF7F5FB009005E0FFF76A
:10173000F1FB0099401A02285AD830698007F6D583
:101740000FE0400840003061FFF7E4FB009005E047
:10175000FFF7E0FB0099401A022849D8306980075A
:10176000F6D42878400765D500200290A06BC00011
:1017700006D4A06B012109070843A0630120029051
:101780005E480168C90511D40168821511430160E2
:10179000FFF7C0FB009005E0FFF7BCFB0099401A83
:1017A000642825D855480068C005F5D5FF20AA68EB
:1017B0000130824203D131690143316111E00121DD
:1017C0008902002A07D005231B029A4203D13269FD
:1017D0000A433261EFE732698243326130698843FC
:1017E0003061A86800280FD0FFF794FB009007E055
:1017F0005EE0FFF78FFB0099411A4148814257D8BC
:1018000030698005F5D50DE0FFF784FB009006E018
:10181000FFF780FB0099411A3948814248D8306966
:101820008005F5D40298002804D0A06B0121090797
:101830008843A063686A002864D00C2F3ED001263C
:1018400036060228206805D0B0432060FFF762FB0F
:1018500005462FE0B0432060FFF75CFB074604E03D
:10186000FFF758FBC01B022822D820688001F7D45C
:10187000E96AA86AE2680843296BFD231B049A43BE
:1018800011430843E060206830432060FFF742FBCB
:10189000054604E0FFF73EFB401B022808D82068FD
:1018A0008001F7D52EE0FFF735FB401B022801D958
:1018B0000320FEBD20688001F5D423E00128F8D084
:1018C000E06801210904AA6A014091420BD10F216D
:1018D0008904EA6A0140914205D103218905084043
:1018E000296B88420ED00120FEBD0000001002408E
:1018F000D83000081800002040100240007000405E
:10190000881300000020EFE7094910B5401E884207
:1019100001D9012010BD074C60610321081F00F0B0
:101920008BFB0020A06107202061002010BD00007B
:10193000FFFFFF0000E000E0F0B502462032137E1A
:10194000012B15D0012717760223537605686C68A2
:10195000AB687026B4430E68496826438024A343CD
:1019600019436E6000688160577600201076F0BDE4
:101970000220F0BD70B5040005D025462035687EF4
:10198000002802D006E0012070BD00202876204605
:1019900000F00AF802206876211D206800F0D4FBD0
:1019A00001206876002070BD00680449884204D197
:1019B0000348816B1022114381637047001000407F
:1019C0000010024070477047F8B502680446D069BD
:1019D0001168936805072D0F5BD0DD07ED0FFF261B
:1019E00021360E402E4367D0C60706D0CE0504D55B
:1019F00001261662E26F3243E2678707022204265D
:101A0000002F06DADF0704D027683A62E76F374312
:101A1000E767470706D5DB0704D023681E62E36F3C
:101A20001343E367020709D520220A402A4305D061
:101A3000236808221A62E36F1343E367E26F002A08
:101A40002FD0800606D5880604D5216E002901D046
:101A500020468847E06F21688968490601D400075D
:101A600024D5204600F03CFC20688168490619D541
:101A70008168402291438160E06E002812D02049A5
:101A80008163E06EFFF750F900280AD0E06E816BA9
:101A900006E0850610D58D060ED5216E1CE0204689
:101AA0008847F8BD2046FFF78EFFF8BD2046FFF7B8
:101AB0008AFF0020E067F8BDC50208D55B0206D5A5
:101AC0000120000510622046FFF77CFFF8BD0306E9
:101AD00005D50B0603D5616E0029E0D1F8BD40069F
:101AE000FCD54806FAD51368204640218B43136085
:101AF000202161670021616600F0BBF9F8BD00009C
:101B0000CD22000810B5040003D0606F002802D079
:101B100007E0012010BD002170200155204600F093
:101B200027F824206067206801684908490001609F
:101B3000204600F03DFC0128ECD0606A002802D06D
:101B4000204600F02DFB206841680922D202914313
:101B50004160206881682A22914381602068016881
:101B6000012211430160204600F080FB10BD0000FF
:101B700010B586B0044614216846FEF708FB1549E7
:101B80002068884224D11448416B012292031143FA
:101B90004163C16A01221143C162C06A69461040B3
:101BA0000590032040020090022001900020029046
:101BB000032003900420049005200007FFF7E8F8B5
:101BC000002211461B20FFF7C9FA1B20FFF7BCFAC1
:101BD00006B010BD0038014000100240F0B5836F20
:101BE000202B54D100290AD0002A08D08568DC01B6
:101BF000A54206D10369002B03D1CB0701D00120F8
:101C0000F0BD034660331E7C012E40D001261E74B9
:101C10004165014640310A834A830022FF2602665D
:101C2000A54204D10569002D13D11A4D0AE07F2782
:101C3000002D09D001263607B5420CD10569002DCB
:101C400005D03F258D8307E00569002D01D08F83E6
:101C500002E08E8300E08A83C267222181670168E7
:101C60008D68012635438D608168A14202D10169EA
:101C700000290AD0084901661A7400680168FF2229
:101C80002132114301600020F0BD0449F3E7022036
:101C9000F0BD0000FF0100005923000801230008E7
:101CA000F8B50068394988426ED1394D2878002846
:101CB0006AD16878AC1E002805D00B27354EFF434B
:101CC000012807D023E0FF208005A0603248E060B3
:101CD000324858E03248FEF7F9FF32213048FEF72B
:101CE00095FF2F48FEF780FE80050DD52C48FEF7A6
:101CF0007DFE80B22080FEF78BFC3146FEF7ABFA0A
:101D00003946FEF7E5FAA060287800283CD16878CB
:101D100002281CD12248FEF7D9FF32212048FEF7C5
:101D200075FF1F48FEF760FE80050DD51C48FEF7C5
:101D30005DFE80B22080FEF76BFC3146FEF78BFA29
:101D40003946FEF7C5FAE060287800281CD168788B
:101D5000032819D11248FEF7B9FF32211048FEF7C7
:101D600055FF0F48FEF740FE80050DD50C48FEF7E5
:101D70003DFE80B22080FEF74BFC3146FEF76BFA49
:101D80003946FEF7A5FA2061F8BD00000038014091
:101D9000020000203333534085EB01409A99793F8C
:101DA00020000020FFB50446406F83B017460D4663
:101DB00020285CD1002D0AD0002F08D0A168C001D6
:101DC000814207D12069002804D1E80702D0012010
:101DD00007B0F0BD204660300290007C012846D05C
:101DE0000298012101740020E06721206067FFF75D
:101DF00091F8264640360190378277820120A1680B
:101E00000003814202D12069002802D02F4600251C
:101E100011E000270FE000228021204600F0DCFBCB
:101E2000002815D1002F15D02168387888627F1CD2
:101E3000708A401E7082708A019B0028069800906C
:101E4000E9D100224021204600F0C6FB002808D03E
:101E50000320BDE728882168C005C00D8862AD1C3D
:101E6000E6E720206067029900200874B0E70220AE
:101E7000AEE77047FEE700001CB50021184800914E
:101E8000164A01910260C16312054260816001221D
:101E9000826302610246C16020321170FF235170DB
:101EA000C233436281621173016381610422416321
:101EB0004261C161FEF79EFD002801D0FEF748FD9A
:101EC000084800900014019069460548FEF742FD5D
:101ED000002801D0FEF73CFD1CBD0000002401409D
:101EE0002000002010000010F0B587B014216846D3
:101EF000FEF74DF91848C16A01252943C162C16A3C
:101F000029400591C26A02210A43C262C06A0324C1
:101F100008400526E4023607059000222146304697
:101F2000FEF7F2FF0D4F002270213846FEF7ECFF5E
:101F30000094002401950294694630460394FEF70C
:101F400027FF70200090029469460195039438465B
:101F5000FEF71EFF07B0F0BD001002400004005065
:101F600010B5144812490160E121C9004160002107
:101F700081600161416181610122C161C2600162D0
:101F8000FFF718F8002801D0FEF7E2FC002109480D
:101F9000FEF7C6FF002801D0FEF7DAFC0021054855
:101FA000FEF7E3FF002801D0FEF7D2FC10BD0000D1
:101FB000005800407C0000201CB500240E4800940E
:101FC0000C49019401600721846041600121446152
:101FD000C160FFF7CFFC002801D0FEF7B9FC0094E8
:101FE000694605480194FFF7A7FC002801D0FEF7D9
:101FF000AFFC1CBD00100040C800002010B50C480C
:102000000A490160E1214902416000218160C1600B
:1020100001618161C1610C22016242614162FFF78D
:1020200071FD002801D0FEF793FC10BD003801407F
:1020300004010020704700008307FF22DB0E9A4056
:102040008907090E994000280BDA0007000F0838AD
:10205000830808489B001818C36993430B43C36166
:102060007047830804489B001B1818689043084376
:102070001860704700ED00E000E400E07047704732
:1020800010B5FFF721F810BD30B599B0342168467E
:10209000FEF77DF814210DA8FEF779F81C2112A88F
:1020A000FEF775F8124801680322D2029143C21468
:1020B0008918016002200090002410200994012555
:1020C000049003956846FFF711FA0F200D908020C9
:1020D0000F900E951094002111940DA8FFF7F4F8BD
:1020E00012A812951494FFF73DF819B030BD000006
:1020F0000070004010480168821511430160C168FA
:102100000E4A1140C16001680D4A114001608168AA
:1021100049084900816001680122920491430160ED
:10212000C168FD2212049143C1600021016105498B
:10213000C003886070470000001002400C40FF8818
:10214000F6FFF6FE00ED00E070B5026801239B0784
:10215000114C124D984203D0A04201D0A84203D1A5
:102160007026B2434E683243984203D0A04201D059
:10217000A84204D103231B029A43CB681A4380234D
:102180009A430B691A4302608A68C26209688162D5
:102190000121416170BD00000008014000140140B0
:1021A00010B5818CC90707D001684A6801235B0418
:1021B0009A43836A1A434A60818C890707D501686C
:1021C0004A6801231B049A43C36A1A434A60818CFC
:1021D000490707D501684A6801239B049A43036BAA
:1021E0001A434A60818C090707D501684A680123B0
:1021F000DB039A43436B1A434A60818CC90607D5B7
:102200000268916801231B039943836B1943916012
:10221000818C890607D501688A6801235B039A438C
:10222000C36B1A438A60818C490612D503685A68C9
:1022300001210905046C8A4322435A60026C8A42D8
:1022400007D10268516803235B059943436C194326
:102250005160818C090607D501684A680123DB04B7
:10226000806C9A4302434A6010BD0000F8B5002616
:102270000446C667FEF74EFE054620680068124F0A
:10228000000709D501212B46002249052046009769
:1022900000F0A2F900280DD12068006840070BD596
:1022A00001212B46002289052046009700F094F971
:1022B000002801D00320F8BD20206067A0676034AB
:1022C00026740020F8BD0000FFFFFF0110B5806AF2
:1022D0000022014640314A834A82FFF774FB10BD59
:1022E00001680A68FF2321339A430A6001688A68FB
:1022F000520852008A6020218167002101667047E0
:1023000010B5014640318B8B846F0268222C04D0BB
:10231000906908210843906110BD526A446D1A40CB
:102320002280426D921C42654A8B521E4A83498B21
:102330000029F1D101680A68FF2321339A430A601A
:1023400001688A68520852008A6020218167002152
:102350000166FFF7A5FC10BD10B5014640318B8B1F
:10236000846F0268222C04D0906908210843906190
:1023700010BD526A1A40436D1A70426D521C42657C
:102380004A8B521E4A83498B0029F1D101680A68A1
:10239000FF2321339A430A6001688A685208520079
:1023A0008A602021816700210166FFF779FC10BD5A
:1023B000F8B504462669A268E769324366691020C9
:1023C00000253E432368324378491E68784F3E40DB
:1023D00016431E6023685A6803263603B243E66834
:1023E00032435A602368A2698B4201D0266A324385
:1023F0009E680B273F02BE4316439E606D4E2368C6
:102400006D4AB3420CD1D2689207920F06D0012ACE
:1024100038D0022A34D0032A20D11EE001201DE04A
:10242000664EB3420AD1D2680C26324026D0042A26
:1024300028D0082A24D00C2A10D10EE08B420DD1CE
:10244000D66803229202164018D001229202B61AD0
:1024500018D0B61A14D0964200D10820564A012648
:10246000403A574FF6038B4236D100280CD0022851
:102470000DD0042812D008281FD11CE00020EDE761
:102480000220EBE70420E9E7FEF7D4FF08E010683C
:10249000C00601D5384605E04A4803E0FEF7EAFFEA
:1024A000002873D0626851005118814205D8110389
:1024B000814202D303E03046F4E7012566E0010ED5
:1024C00006025008002330185941FDF729FE032168
:1024D0000902411A3C4A55E0E169B14232D1030098
:1024E00000F0DBF809070A0D06250606062B060094
:1024F000E3E7FEF79FFF1CE0FEF7ACFF19E0106872
:102500006168C00602D54808304A01E0304A4808F0
:102510008018FDF7EFFD80B201462E4A1039914236
:10252000CBD8511C01400007400F08432CE0FEF7B8
:10253000A1FF616840004A08EAE761680122480893
:102540001204E5E7030000F0A8F809070A0D0626C3
:102550000606062C0600B0E7FEF76CFF1DE0FEF74E
:1025600079FF1AE010686168C00602D54808C019F2
:1025700002E014484A081018FDF7BCFD80B201467D
:10258000144A1039914298D82168C860002020660A
:1025900060662846F8BDFEF76DFF61684A0880183E
:1025A000EAE7616848088019E6E700000048004053
:1025B000F369FFEF00380140401002400044004042
:1025C00000093D000024F400FFFC0F0000127A0017
:1025D0000048E801EFFF0000FFB581B017460E4646
:1025E00004460A9D09E0681C07D0FEF793FC049995
:1025F000401AA8420CD8002D0AD02068C169304684
:10260000884318D00020B842EDD0002005B0F0BDBE
:1026100020680168FF22A13291430160206881682F
:1026200049084900816020206067A067002060346D
:1026300020740320EAE70120E5E7000010B5024816
:10264000FFF7C2F910BD0000040100200FB410B55F
:1026500003A9044B044A029800F0F6F810BC08BC29
:1026600004B01847852F00081C0000202021020C10
:1026700001D010211046020A01D010460839020983
:1026800001D01046091F820801D01046891E420859
:1026900001D0881E7047081A704730B47446641E13
:1026A0002578641CAB4200D21D46635D5B00E318D5
:1026B00030BC184702E008C8121F08C1002AFAD12E
:1026C00070477047002001E001C1121F002AFBD1B2
:1026D00070470000F0B51FB486B00998089A030D42
:1026E0000021024314D05148514A18185043051490
:1026F0001198012810981AD0281A401C00264D4F16
:102700004D49009601910490002812DA444211E0EC
:102710001198012449A3012801D11098C1430698BA
:10272000119A84600360C26041600BB0F0BD40420A
:10273000E4E70446210500203F4A001C5141039173
:10274000029012E0E00707D032463B46019900981C
:10275000FDF77EFE0191009032463B461046194639
:10276000FDF776FE06460F466410002CEAD1049869
:10277000039B0028029A0999089806DAFDF768FE7B
:10278000019B009AFDF764FE05E0FDF7C9FE019B81
:10279000009AFDF7C5FE04460E460022284BFEF7C0
:1027A0006DF803D80020C043014607E00022254B06
:1027B00020463146FDF798FDFEF740F8102409E069
:1027C000002C0ADB0A220023FDF7AAFC079B30320B
:1027D0001A55641E02460A43F2D11122641C079B5B
:1027E000121B1C19119B012B03D0012308430ED18E
:1027F0000AE0084304D0112010900020119077E7E0
:102800001098151A6D1E0BE01098824202DD00230D
:102810006D1C03E0824201DA00236D1E002BEED016
:10282000069811998260C16030C07EE701FCFFFF0D
:10283000104D0000000014400000F03F3000000088
:102840000000F0430000E03FFFB597B006460025CA
:102850001BE2252876D100242746F749049400E09E
:102860000443761C32780120203A90400842F7D188
:1028700030782A280ED002223078014630390929D2
:1028800016D804990A235943303940181443761C4A
:102890000490F1E7189802C804911890002904DA0E
:1028A0000120400304434842049002200443761C64
:1028B00030782E2814D1042004437078761C2A28FE
:1028C00009D11898761C80C8189009E00A214F4356
:1028D000303FC719761C3078014630390929F5D9BF
:1028E00030786C2810D006DC4C281AD068280ED01E
:1028F0006A2817D104E0742813D07A2812D110E086
:102900000120400504430CE00121090501E00321F9
:1029100009050C437178814203D101200005241878
:10292000761C761C307866280BD013DC58287DD0B6
:1029300009DC00287BD04528F6D04628F4D047286B
:102940001AD1A9E118E0632835D0642870D0652831
:1029500012D1A1E170286CD008DC6728F1D0692879
:102960007DD06E280DD06F2806D1BCE073282ED004
:10297000752873D0782859D01A9A199990476D1CE8
:1029800082E16002400F022809D003280DD00428FC
:10299000189801680DD00D60001D189074E118980A
:1029A000EA1701680D604A60F6E7189801680D8023
:1029B000F2E70D70F0E718986A4601781172001D71
:1029C00018900020507202A80090012005E018988D
:1029D00002C8189000200091C04361070ED5002165
:1029E00001E00199491C0191B94213DA8142F8DBF7
:1029F000019A0099895C0029F3D10BE0002101E0E4
:102A00000199491C01918142FADB019A0099895C84
:102A10000029F5D1019904981A9B471A2146384696
:102A2000199A00F099FA4019019903E051E030E158
:102A300015E050E0451807E0009800990078491C1F
:102A400000911A9A199990470198401E0190401CD4
:102A5000F2D1214638461A9B199A12E137E00A2032
:102A60000021009001916002410F022907D0189ABD
:102A700001CA1892C2179446032908D00AE0189890
:102A8000C01DC108C90005C91891944607E000B2ED
:102A9000C2179446042902D140B2C1178C460022C5
:102AA0006146944506DA0A460021404291418C462F
:102AB0002D2102E0210504D52B216A461173012145
:102AC00003E0E10701D02021F7E7029156E00A2058
:102AD0000AE0102008E010200090002104200443A8
:102AE0000191082703E00820002101910090600275
:102AF000410F022907D0189A01CA18920022944661
:102B0000032908D008E01898C01DC108C90005C9EC
:102B10001891944603E080B2042900D1C0B200218C
:102B2000029121072AD531780D91702906D0009A9B
:102B30001021019B4A401A4305D00EE040216A460D
:102B40001173012108E06146014306D030216A4635
:102B500011730D99517302210291009A0821019B72
:102B60004A401A430AD16146014301D1610705D5A4
:102B700030216A46117301217F1E02913178582954
:102B800004D02EA10E910DA90D910DE030A1F9E711
:102B90006146019B009AFDF7C3FA0E9B8C469B5C35
:102BA0000D9A521E0D92137061460143F0D10D989B
:102BB00005A9081A20300190600703D50120000400
:102BC000844300E001270198874201DD381A00E0C4
:102BD0000020019900904118029809180498401AA1
:102BE0000490E00306D421461A9B199A049800F039
:102BF000B3F94519002706E003A81A9AC05D199990
:102C000090476D1C7F1C02988742F5DBE0030CD5D2
:102C100021461A9B199A049800F09EF9451904E080
:102C20001A9A3020199990476D1C0099481E0090FF
:102C30000029F5DC1FE000000928010030313233A3
:102C400034353637383961626364656600000000E8
:102C500030313233343536373839414243444546D2
:102C6000000000000D980D990078491C0D911A9AEA
:102C7000199990476D1C0199481E01900029F1DCBB
:102C80004DE100F059F94519761C3078002800D044
:102C9000DFE528461BB0F0BD600700D40627189872
:102CA000C01DC108C90048680A680831C30FDB07A6
:102CB0001891190001D09CA108E0210501D59BA124
:102CC00004E0E10701D09AA100E09AA1430010912D
:102CD00030785B0865280CD006DC452809D04628EA
:102CE0001DD0472841D141E0662818D067283CD143
:102CF0003CE00021112F01DB112000E0781C019144
:102D0000009008A911A8FFF7E5FC1399059100218F
:102D1000119A15927F1C12980197009150E00120A2
:102D2000C00703900120019008A9009711A8FFF7A0
:102D3000D1FC139A149905920022119B00921298CB
:102D40001593059A0192002901D0104602E0791CE2
:102D500040180190381A01D5019804E04042401E05
:102D60000090781C0190C01B029043E0012F00DA14
:102D700001270021112F01DD112000E038460191CB
:102D8000009008A911A8FFF7A5FC13990591119AC5
:102D90000021129815920091019721070CD40599F2
:102DA000B94201DB019900E00191012904DD159A86
:102DB000491E515C302906D0B84201DA011D05DAFE
:102DC0000121029115E00199491EEDE7002805DC7B
:102DD0000099411800910199091A03E0019A411CD8
:102DE000914200DD01910099401A401C029001209F
:102DF000C0070390200706D402990198814202DBA4
:102E00000020C043029000206946C87707AF012127
:102E100003980337C907884224D0022011902B2041
:102E20001290039800280CDA404203902D20129053
:102E300007E00A210398FDF75DF930317F1E03900A
:102E400039701199481E11900029F2DC039800286E
:102E5000EFD1791E12980870307820210840453053
:102E6000BF1E387006A8C01BC01D039010980078C4
:102E7000002800D00120019941180298C0170918B4
:102E8000039809180498401A401E0490E00306D4E1
:102E900021461A9B199A049800F05EF8451910987B
:102EA0000078002803D01A9A199990476D1CE00306
:102EB00024D521461A9B199A049800F04DF845191B
:102EC0001CE00098002807DB00990598884203DD84
:102ED0001598405C199901E0199930201A9A904789
:102EE00000986D1C401C00900298401E0290002823
:102EF00004D11A9A2E20199990476D1C0199481EE9
:102F000001900029DDDC05E038781A9A7F1C1999B8
:102F100090476D1C0399481E03900029F4DC21465C
:102F20001A9B199A0498ACE62D0000002B000000B3
:102F30002000000000000000F8B5044600251E46F1
:102F40001746880404D405E039462020B0476D1C9C
:102F5000641EF9D52846F8BDFFB50446002581B0AA
:102F60001E46C80301D5302700E02027880404D579
:102F700005E038460399B0476D1C641EF9D5284614
:102F800005B0F0BD01B5044B012269460348FEF7C8
:102F900009FF009808BD0000FFFF000004010020A9
:102FA00008B5FEF799F8FFF76FF8FEF79DFFFFF7FA
:102FB00025F8FFF701F8FEF75FFFFEF7D1FF364C6B
:102FC000364F3748FDF782FE32213548FDF71EFEA9
:102FD0003348FDF709FD800553D53148FDF706FD5F
:102FE00080B22080FDF714FB2E4D2946FDF733F902
:102FF0000B26F6433146FDF76BF9FDF710FB024651
:103000000B4629A0FFF722FB2088FDF701FB29468C
:10301000FDF721F93146FDF75BF90546A168FDF79B
:103020002FFBA1682846009108D2FDF70CF9FDF7A7
:10303000F6FA05460E460099E06807E0FDF703F949
:10304000FDF7EDFA05460E4621690098FDF7FBF8FD
:10305000FDF7E5FA02460B4600203946FDF760FA17
:103060002A463346FDF7F4F90022144BFDF7E7F941
:10307000FDF7E9FAFDF7D3FA02460B4610A0FFF779
:10308000E5FA05490422891C1148FEF7A7FD1148FD
:10309000FDF770FE95E700000000002000000840EA
:1030A0002000002033335340766F6C7461676520D5
:1030B0003A2025312E3366560D0A000000001C40D0
:1030C0005048203A2025312E31660D0A00000000BC
:1030D0000401002010270000000000000000000094
:1030E0000102030406070809030406080C1018204F
:1030F0003000000000010203040000001C31000841
:103100000000002020000000B42600083C31000828
:103110002000002068050000C42600080000000010
:10312000000000000000C03F85EB01409A99793F04
:0C31300000000000000020000000000073
:04000005080000C12E
:00000001FF
